:020000040000FA
:020000000528D1
:08000800052803138312850192
:1000100007309F0083161030850001308600831260
:10002000A001A101A201A3014120051E102806186C
:1000300014283B2006181428A00A0A302002031DA9
:100040003428A001A10A0A302102031D3428A1018D
:10005000A20A0A302202031D3428A201A30A0A3090
:100060002302031D3428A3013B20061C34283B2017
:10007000061C342814280630A5004120A50B3D2875
:100080000800FE3086000730850023085E207720B8
:10009000FE3086000B30850022085E207720FE307F
:1000A00086000D30850021085E207720FE30860016
:1000B0000E30850020085E2077200800A60003107F
:1000C000260D820780307528F23075284830752853
:1000D0006030752832307528243075280430752832
:1000E000F030752800307528203086000800643014
:0800F000A400A40B792808000C
:02400E00223F4F
:00000001FF
